:0800000023C051C0FDCFFCCF6D
:10000800FBCFFACFF9CFF8CFF7CF70C0F5CFF4CF49
:10001800F3CFF2CFF1CFF0CFEFCFEECFEDCFFFFFA1
:10002800787878787878787807000D007800DE009E
:10003800FF000A006201260001006C013000000088
:10004800F894EE27ECBBF1E0FBBFEBBFE5BFF8E1AE
:10005800F1BDE1BD8DE0A2E0BB27ED938A95E9F7FC
:1000680080E094E0A0E6ED930197E9F7EAE3F0E099
:1000780085919591009761F0A591B591059015909E
:10008800BF01F00105900D920197E1F7FB01F0CF58
:10009800EFE5EDBFE4E0EEBFC0E6D1E04DC0AA93C6
:1000A800EA93EFB7EA93E0E0E2BFE0916001EF5F27
:1000B800E0936001E0916C01A0916001EA1788F477
:1000C800E0E0E0936001E0916101EF5FE09361019E
:1000D800A0916101AA3018F0E0E0E0936101689412
:1000E80020F8E991EFBFE991A9911895EA93E0E02A
:1000F800E0936001E9911895E4EAE6BF3ED1F1F397
:100108003FD1E830B9F4E0E53ED137D1F1F338D149
:10011800E83181F4EFEA37D130D1F1F331D1E83267
:1001280049F4E88130D129D1F1F32AD1E83211F428
:10013800E4E9E6BF21960895EFE3E8BBE0E0E7BB1A
:10014800EFE0E5BBE0E0E4BBEBEFE2BBE0E0E1BB06
:10015800E4E0E3BFE0E0E2BFEFBDEEBDEDBDECBD26
:10016800E7BDE6BDEBBDEABDE9BDE8BDE2BDE5BD65
:10017800E4BDE3BDEBB7E064EBBFE3E0E5BFE0E47B
:10018800EABFE1E0E9BFE0E8E8B9E0E0E0BFE1B9F3
:10019800ECE0E0B9E0E0E2B9E4E0E6BFE0E0859950
:1001A800E1E0E13010F0E7E001C0E9E0E0936C0144
:1001B800EEE1E1BDEEE0E1BDEAD0EA939DDF78949F
:1001C800A895E8E3F0E0E491E0936201A3E6B1E0EA
:1001D800E8E3F0E0E491EC93E0E09899E1E0E130C5
:1001E80028F0E0E09999E1E0E13008F403C0A4E6E2
:1001F800B1E0D1D0989903C0A4E6B1E0CFD09999E5
:1002080003C0A4E6B1E0CFD0E0E09A99E1E0E130A4
:1002180028F0E0E09B99E1E0E13008F403C0A5E6AE
:10022800B1E0B9D09A9903C0A5E6B1E0B7D09B99DF
:1002380003C0A5E6B1E0B7D0E0E08099E1E0E130A5
:1002480028F0E0E08199E1E0E13008F403C0A6E697
:10025800B1E0A1D0809903C0A6E6B1E09FD0819912
:1002680003C0A6E6B1E09FD0E0E08699E1E0E13086
:1002780028F0E0E08799E1E0E13008F403C0A7E660
:10028800B1E089D0869903C0A7E6B1E087D0879905
:1002980003C0A7E6B1E087D0E0E0B099E1E0E13043
:1002A80028F0E0E0B199E1E0E13008F403C0A8E605
:1002B800B1E071D0B09903C0A8E6B1E06FD0B199B0
:1002C80003C0A8E6B1E06FD0E0E0B299E1E0E13028
:1002D80028F0E0E0B399E1E0E13008F403C0A9E6D2
:1002E800B1E059D0B29903C0A9E6B1E057D0B399AB
:1002F80003C0A9E6B1E057D0E0E08399E1E0E1303E
:1003080028F0E0E08499E1E0E13008F403C0AAE6CF
:10031800B1E041D0839903C0AAE6B1E03FD0849907
:1003280003C0AAE6B1E03FD0E0E0B499E1E0E130F3
:1003380028F0E0E0B599E1E0E13008F403C0ABE66D
:10034800B1E029D0B49903C0ABE6B1E027D0B599A4
:1003580003C0ABE6B1E027D0E0E020FCE1E0E1300B
:1003680050F0E89420F8E0916101F0E0EE59FE4F7A
:10037800E081EA93C1DE24CFFFCFE6B7E0780895A5
:10038800E1B1E87F0895E3B9E4E8E6BF0895E4E35E
:10039800F0E0E4910895FBDFEC930895E6E3F0E0E4
:1003A800E491EC930895E2E3F0E0E491EC9308958E
:00000001FF
